:020000040000FA
:0400000024EF01F0F8
:10000800D8CF00F0E0CF01F0026EE9CF03F0EACFDD
:1000180004F0FACF05F0FBCF06F09DA816D09EA8F5
:1000280014D06750E96E020E6824EA6EEFCFADFF78
:100038007888672A000E6822676605D0020E686213
:1000480002D0676A686A6F4E9D98F2A815D0F2A22E
:1000580013D0F292F29878A48B947786E80ECF6E3C
:10006800900ECE6E9E90CD8077A806D0779877A216
:1000780003D00D0E7464742A9DAA67D09EAA65D019
:100088007786E80ECF6E900ECE6E9E90CD80ABA296
:1000980003D0AB98AB8859D0ABA415D0AE50E20EC4
:1000A800CF6EB40ECE6E9E90CD8077AC05D0779C87
:1000B800AC9A4A0EAF6E49D078A847D0AC9A7898D7
:1000C800778E779242D001EE80F06650E926AECF67
:1000D800EFFF77AC05D0779CAC9A4A0EAF6E2BD069
:1000E80078A829D06D50E96E020E6E24EA6EEFCF23
:1000F80079F001EE80F06650E926EF50791811E0AA
:10010800AC9A7898778C778E77927C0EAF6E9D98A4
:10011800AD6AAC8AE20ECF6EB40ECE6E9E90CD80E4
:100128000AD06D2A000E6E226D6605D0020E6E6230
:1001380002D06D6A6E6A5F0E716007D077BC05D019
:10014800662A600E666201D0666A9EA051D09E90B3
:1001580077A64AD07796F292F28878A48B8474C0F6
:100168007AF07A467A46F9507A44F926E80ECF6E44
:10017800900E36D0E90ECF6EBC0E32D0EA0ECF6E9E
:10018800E80E2ED0EC0ECF6E140E2AD0ED0ECF6EE8
:10019800400E26D0EE0ECF6E6C0E22D0EF0ECF6E34
:1001A800980E1ED0F00ECF6EC40E1AD0F10ECF6E80
:1001B800F00E16D0F30ECF6E1C0E12D0F40ECF6ECA
:1001C800480E0ED0F50ECF6E740E0AD0F60ECF6E16
:1001D800A00E06D0F70ECF6ECC0E02D0F80ECF6E62
:1001E800CE6ECD80778804D077A802D07798CD904E
:1001F8009EA218D09E92572E15D0050E576E2682B5
:10020800582E03D0020E586E2684592E0BD0140E89
:10021800596E26865A2E06D00A0E5A6E26885B2EEE
:1002280001D05B6E05C0FAFF06C0FBFF03C0E9FF03
:1002380004C0EAFF025001C0E0FF00C0D8FF100070
:1002480091EC10F0C4EC10F011EC11F0000144EC4A
:1002580011F00400D180F28CF28ECA8477B24FD0AC
:1002680077AE05D0779E6BC067F06CC068F06750BA
:10027800695C076E68506A58086E08AE02D0020EB4
:100288000826075008104DE06750E96E020E6824F2
:10029800EA6EEFAE2BD0096A020E0A6E67C00BF049
:1002A80068C00CF007C00DF00E6A0F6E76EC09F00E
:1002B8006F6E6F5036E0FF0A03E101EC0EF031D0AB
:1002C8006750E96E020E6824EA6EB20EEF6203D040
:1002D800070E746E01D0746A67C06BF068C06CF06A
:1002E80067C06DF068C06EF077821BD001EC0EF02D
:1002F8000706000E085A07500810C6E112D0ACA233
:1003080006D06F6604D0746A789877920AD077B866
:1003180008D077BC06D078A604D077B602D09D88DE
:10032800AC8A77B430D06550665C076E07AE02D0F1
:10033800600E072607C071F0075255E001EE80F005
:100348006550E926EFAE1AD0800E096E010E0A6ECE
:1003580065C00BF00C6A0BBE0C0607C00DF0600EF2
:100368000E6E0F6A76EC09F0706E70503CE0FF0A72
:1003780003E1F6EC0DF037D0778435D0F6EC0DF0CC
:10038800072EDCD730D001EE80F06550E926EF501B
:10039800830A0BE0330A0CE0010A14E0030A16E0B2
:1003A800060A18E05B0A19E01BD0CBEC0DF01AD056
:1003B800000ED6EC0BF00FC008F010C009F094EC5A
:1003C8000AF010D0010ED6EC0BF00CD0020ED6ECD1
:1003D8000BF008D049EC0FF005D045EC0EF002D038
:1003E800F6EC0DF0779410EEB0F0076A080E07608F
:1003F800A1D0E650E6BE9CD0EA6A470E0724E96E13
:10040800EF50D8B495D024EE00F0200E0702F35038
:10041800D9260C6A010E086E0852D8B480D0EA6A50
:10042800470E0724E96E0850EF1473E0EA6A470E96
:100438000724E96E081CEF16DECF0BF0DECF09F0BB
:100448000F0E09140A6E0938070B096E095006E0E9
:10045800010A04E0030A02E0010A5DE109C00EF0A6
:100468000AC00FF00BC010F00CC011F007C012F05A
:1004780008507BEC08F006E3EA6A800E0724E96E70
:100488000850EF12095203E0020E09620CD00A521A
:100498000AE0EA6A2F0E0724E96E0850EF1403E118
:1004A800020ED92638D0DE50DEBE35D0D8900B32B9
:1004B800D8900B32030E0B14010A05E0030A11E071
:1004C800010A20E028D0EA6A2F0E0724E96E0850B6
:1004D800EF1421E0EA6AA00E0724E96E0850EF1233
:1004E8001AD0EA6A2F0E0724E96E0850EF1413E1B8
:1004F800E550E6BC10D0EA6AA00E0724E96E085061
:10050800EF1209D0EA6AA00E0724E96E0850EF122C
:1005180002D0040ED9260C2AD89008367DD707C0F9
:1005280024F0EA6A2F0E0724E96EEF5000EC10F071
:10053800072A5CD726A275D02692040026AE06D0DC
:100548005D2E04D0269E000E48EC07F081B008D03E
:1005580078A60DD0722A140E726209D0789607D048
:10056800726A78B604D0736602D0010E736E735245
:100578000EE0732A330E73620AD0736AF29E9D9856
:10058800F292F288AB889E9A9D8AF28E788610EE57
:10059800B0F0076A080E076044D0E650E6AE3FD0D8
:1005A800EA6A370E0724E96EEFCF09F00750ECEC42
:1005B8000FF00A6EEA6A2F0E0724E96E0AC0EFFFF1
:1005C800EA6A4F0E0724E96EEFCF0CF0EA6A800E54
:1005D8000724E96EEFCF0DF00A5009180B6E010ED3
:1005E800086E085216E008500D1410E10C500B1458
:1005F80008140CE0EA6A370E0724E96E0850EF1A6F
:10060800EA6A470E0724E96E0850EF12D8900836B8
:10061800E8D7EA6A4F0E0724E96E0BC0EFFF072AF6
:10062800B9D726A4A4D326940A6A080E0A6054D11E
:10063800EA6A980E0A24E96EEF50D8B44BD124EE3A
:1006480000F0200E0A02F350D9260D90076A010E19
:100658000B6E0B52D8B433D1EA6A980E0A24E96EAD
:100668000B50EF14D8B425D1DECF09F0DDCF0CF054
:100678000C38070B086E01EE00F0080E0A02F35062
:100688000724D890E834E926EE06000EEE5A01EE6B
:1006980000F0080E0A02F3500724D890E834E9263F
:1006A800EE50EE10D8A405D1E26AD8900A34B10F02
:1006B800E16EE7BED2D0E7AA17D0050ED9260C38CE
:1006C800F00B0C6E0F0EDF140C26050ED95E08C059
:1006D8000EF00CC00FF007C010F00AC011F00B505C
:1006E800EBEC07F00D80E5D0EA6AA80E0A24E96E63
:1006F8000B50EF1433E0EA6A980E0A24E96E0B1CDB
:10070800EF16EA6A800E0A24E96E0B50EF1413E024
:1007180008C00EF00F0E0C140F6E106A07C011F00F
:100728000AC012F00B507BEC08F0EA6A800E0A242B
:10073800E96E0B1CEF16EA6AA80E0A24E96E0B1C78
:10074800EF16EA6A270E0A24E96E0B50EF12EA6ADE
:10075800A00E0A24E96E0B50EF12ABD00850020A23
:1007680003E0030E08621CD0EA6A980E0A24E96EB8
:100778000B1CEF1608C00EF00F0E0C140F6E106A4B
:1007880007C011F00AC012F00B507BEC08F006E32A
:10079800EA6A800E0A24E96E0B50EF120D8028D009
:1007A800085202E0082C24D0EA6A980E0A24E96E5E
:1007B8000B1CEF16EA6A800E0A24E96E0B1CEF1672
:1007C800DFBC08D0EA6A2F0E0A24E96E0B1CEF166C
:1007D8000D800ED0EA6A370E0A24E96E0B50EF142A
:1007E80007E1EA6A2F0E0A24E96E0B1CEF160D804A
:1007F800030ED926DFBE2ED0D8900932D890093200
:100808000914010A05E0030A11E0010A1DE022D0DB
:10081800EA6A2F0E0A24E96E0B50EF141BE0EA6A0D
:10082800A00E0A24E96E0B50EF1214D0EA6A2F0EBC
:100838000A24E96E0B50EF140DE1EA6AA00E0A24AF
:10084800E96E0B50EF1206D0EA6AA00E0A24E96E90
:100858000B50EF12030ED95E2CD0EA6A980E0A24C8
:10086800E96E0B1CEF16EA6A270E0A24E96E0B5094
:10087800EF12EA6AA80E0A24E96E0B50EF1413E08F
:10088800EA6AA80E0A24E96E0B1CEF16EA6AA00EA3
:100898000A24E96E0B50EF12EA6A800E0A24E96E08
:1008A8000B1CEF1606D0EA6A470E0A24E96E0B50B5
:1008B800EF12040ED926072AD8900B36CAD60DA0F7
:1008C80009D00AC024F0EA6A2F0E0A24E96EEF5014
:1008D80000EC10F00A2AA9D610EEB0F00D6A080E46
:1008E8000D607ED1D8900D340F6EE6CF07F0E6CFBD
:1008F80008F008AE73D16750695C096E68506A5891
:100908000A6E0AAE02D0020E0A26EA6A470E0D24C3
:10091800E96EEF50D8B462D10ABE06D0C00E095CA9
:10092800010E0A58D8B05AD124EE00F0200E0D025C
:10093800F350D926040ED95E000EDA5A1068010E5B
:100948000E6E0E52D8B44AD1040ED926000EDA2201
:10095800102AEA6A470E0D24E96E0E50EF14D8B437
:100968003AD1EA6A470E0D24E96E0E1CEF16DECF67
:100978000BF0DDCF0CF01290EA6A370E0D24E96E09
:100988000E50EF14D8A41280089612B008860B38BF
:10099800030B37E178B01FD1089812B00888EA6ACB
:1009A800270E0D24E96E0E50EF14D8B48BD0EA6AE6
:1009B800270E0D24E96E0E1CEF160896EA6A3F0E04
:1009C8000D24E96E0E50EF140888D8B408980BC0AF
:1009D80013F01980199207C014F008C015F01050D0
:1009E800EDEC09F0EA6AA00E0D24E96E0E50EF1442
:1009F800D8A4F1D0EA6A800E0D24E96E0E1CEF1619
:100A0800EAD00C38070B5EE178B05CD0EA6A270EB2
:100A18000D24E96E0E50EF1416E0EA6A270E0D2435
:100A2800E96E0E1CEF16EA6A880E0D24E96E0E5068
:100A3800EF14D880D8B4D89003E212B0CCD042D00A
:100A480012B040D0C8D0EA6A980E0D24E96E0E5054
:100A5800EF1422E1EA6A880E0D24E96E0E1CEF16E7
:100A680012A010D00E50EF12030E0B14030A2AE046
:100A78000CC013F010C014F00DC015F00E5041EC6E
:100A880009F0A9D00CC013F010C014F00DC015F077
:100A98000E5041EC09F09FD0EA6A880E0D24E96EE9
:100AA8000E50EF14D880D8B4D89003E212B003D017
:100AB80009D012B007D0EA6A980E0D24E96E0E1C10
:100AC800EF1689D0030E0B14010A07E0030A08E0A9
:100AD800010A08E0030A54E005D012B003D050D050
:100AE80012B04ED00B38030B40E1EA6A980E0D2481
:100AF800E96E0E50EF146FE1EA6A3F0E0D24E96EBD
:100B0800EFCF11F008AC03D00E50111A07D010A087
:100B180003D00E50111202D00E1C11160E501114D3
:100B28000888D8B40898EA6A3F0E0D24E96E11C007
:100B3800EFFF0C38070B020A09E10CC013F010C0D4
:100B480014F00DC015F00E5098DB08D0200E136E6F
:100B580010C014F00DC015F00E508FDB0886EA6A3D
:100B6800800E0D24E96E0E50EF120BC013F01980A1
:100B7800199207C014F008C015F01050EDEC09F0F8
:100B8800D8900B32D8900B32030E0B14010A07E0F1
:100B9800030A08E0010A08E0030A1DE005D012B0C4
:100BA80003D019D012B017D0EA6AA00E0D24E96E4E
:100BB8000E50EF12030ED926000EDA22DF38030B8F
:100BC80006E1EA6A800E0D24E96E0E50EF12030E5C
:100BD800D95E000EDA5AD8900E36B3D60D2A7FD6D3
:100BE8000E6A080E0E60B3D06750695C096E6850D3
:100BF8006A580A6E0AAE02D0020E0A26EA6AA00EE7
:100C08000E24E96EEF50D8B4A0D00ABE06D0E00E8C
:100C1800095C010E0A58D8B098D0E26AD8900E3410
:100C2800B10FE16E24EE00F0200E0E02F350D9262B
:100C3800116A010E0F6E0F52D8B487D0EA6A470EB8
:100C48000E24E96E0F50EF147AE1EA6AA00E0E2422
:100C5800E96E0F50EF1473E0E7AE07D0EA6A980E1A
:100C68000E24E96E0F50EF146DE1EA6AA00E0E240F
:100C7800E96E0F1CEF16DECF0BF0DECF0DF0DECFE6
:100C880007F0DECF08F0040ED95E08C00CF0089813
:100C9800EA6A370E0E24E96E0F50EF14D8A40888BC
:100CA8000C38030B42E1EA6A270E0E24E96E0F5056
:100CB800EF1408E0EA6A270E0E24E96E0F1CEF16FF
:100CC800089825D0E7AE14D00B38030B020A10E1C0
:100CD800EA6A3F0E0E24E96E0F1CEF16E7AC08D047
:100CE80008A806D0EA6A3F0E0E24E96E0F50EF12EC
:100CF800200E136E11C014F00EC015F00F50BDDA9F
:100D08000888EA6AA80E0E24E96E0F50EF12E7AEC3
:100D180007D0EA6A3F0E0E24E96E0F50EF1401D097
:100D2800000E000A088AD8B4089A0CC013F019807B
:100D3800198207C014F008C015F011504ADB040EE0
:100D4800D926112AD8900F3676D70E2A4AD778A0F6
:100D58000ED0076A080E076007D0EA6A470E072414
:100D6800E96EEF10072AF6D7FF0AD8A4789026A6CE
:100D780059D026965E520DE05E060F0E5E1409E10C
:100D88005E3A5E060F0E5E1403E0140E7DD85E8A8E
:100D98005E3A5F5206E05F2E04D0640E75D80A0EE4
:100DA8005F6E78A223D075060F0E75141FE1753A91
:100DB8000F0E7514076E080E076014D0010E086E2A
:100DC800075005E0096ED8900836092EFCD7085060
:100DD800601406E0EA6A470E0724E96EEE68788038
:100DE800752A01D07892753A0A0E751282B219D016
:100DF8005C2A78B407D00A0E5C620BD07884010EA6
:100E08005F6E07D0020E5C6204D078945F6A650E4C
:100E18005C6E640E5C6203D0D19000EF00F00001BC
:100E280001D05C6A26A832EF01F0269826AA32EF94
:100E380001F05B04076E080E076032EF01F0E26A0A
:100E4800D8900734B10FE16EE7AE0FD00750612498
:100E5800196E000E62201A6EEA6A3F0E0724E96EC8
:100E6800EF5036EC10F032EF01F007506124196EA4
:100E7800000E62201A6EEA6A370E0724E96EEF50F8
:100E880036EC10F032EF01F0246E245205E024C055
:100E98005DF0268E8B9001D08B8012001C6E010EA7
:100EA800EA6E1BC0E9FF1C461C461C44060FF924C9
:100EB800D8B0FA2AF96EEF6A000E00003BD00A0E8D
:100EC800EF6E000E37D0140EEF6E000E33D0230EE7
:100ED800EF6E000E2FD0320EEF6E000E2BD0410EAB
:100EE800EF6E000E27D0500EEF6E000E23D0640E6A
:100EF800EF6E000E1FD07D0EEF6E000E1BD0960E0B
:100F0800EF6E000E17D0C80EEF6E000E13D02C0E29
:100F1800EF6E010E0FD0900EEF6E010E0BD0F40E97
:100F2800EF6E010E07D0580EEF6E020E03D0200EA2
:100F3800EF6E030EEC6E1200196E010EEA6E18C009
:100F4800E9FF19461946F9501944F926E80EEF6EDB
:100F5800030E3BD0DC0EEF6E050E37D0D00EEF6ED1
:100F6800070E33D0B80EEF6E0B0E2FD0A00EEF6E1B
:100F78000F0E2BD0880EEF6E130E27D0700EEF6E6B
:100F8800170E23D0280EEF6E230E1FD0E00EEF6E43
:100F98002E0E1BD0500EEF6E460E17D0C00EEF6E01
:100FA8005D0E13D0300EEF6E750E0FD0A00EEF6EE3
:100FB8008C0E0BD0100EEF6EA40E07D0800EEF6EC5
:100FC800BB0E03D0600EEF6EEA0EEC6E1200126ECE
:100FD800EA6A2F0E1124E96EEFCF14F0105005E0E5
:100FE800176ED8901432172EFCD7030E14160F1450
:100FF800146214D026900FB426802F0E1124246E6C
:1010080012501BEC10F026900FB626802F0E1124DC
:10101800246ED89012341BEC10F013D026900FB029
:1010280026802F0E1124246E12501BEC10F02690EF
:101038000FB226802F0E1124246ED89012341BEC88
:1010480010F011C024F0EA6A2F0E1124E96EEF5057
:1010580000EC10F00F380F0B0F6E080E1102F35052
:101068001024136EEA6A980E1124E96E121CEF160A
:101078000E50020A03E0010A19E02FD0D890133469
:101088001B6E0F500BDF01EE00F0D8901334E926E9
:10109800EECF15F0EECF16F0155016101EE0EA6AE6
:1010A800980E1124E96E1250EF1217D0D89013340D
:1010B800186E0F5041DF01EE00F0D8901334E92686
:1010C800EECF15F0EECF16F01550161006E0EA6ACE
:1010D800980E1124E96E1250EF1201EE00F0D8902C
:1010E8001334E92615C0EEFF16C0EEFF1200136E8A
:1010F8000E5202E00E2C0BD010BC09D0EA6A980EF2
:101108001224E96E1350EF1402E0D8901200EA6A34
:10111800370E1224E96E1350EF14D8B48FD0080E8E
:101128001202F3501124146E0E5203E0020E0E62E6
:1011380006D0D89014341B6E0F50B0DE0AD00E4C77
:1011480003D0030E0E6205D0D8901434186E0F50D9
:10115800F3DE01EE00F0D8901434E926EECF16F055
:10116800EECF17F00E50020A07E0010A10E0030A5A
:1011780037E0010A40E060D01650171008E1EA6A2B
:101188002F0E1224E96E1350EF12D8901200EA6A5B
:10119800980E1224E96E1350EF144EE1EA6AA80E75
:1011A8001224E96E1350EF1405E0090E165E000EC6
:1011B800175A06D0EA6A2F0E1224E96E1350EF1A56
:1011C80001EE00F0D8901434E92616C0EEFF17C0DF
:1011D800EEFFEA6A980E1224E96E1350EF122CD033
:1011E8001650171008E1EA6A2F0E1224E96E135000
:1011F800EF12D8901200EA6AA80E1224E96E135072
:10120800EF1405E0090E165E000E175A06D0EA6ABA
:101218002F0E1224E96E1350EF1201EE00F0D89051
:101228001434E92616C0EEFF17C0EEFFEA6A980EDE
:101238001224E96E1350EF12D88012000E50020AE1
:1012480007E0010A05E0030A09E0010A07E013D0F4
:10125800EA6A980E1224E96E131CEF16EA6A980ED1
:101268001224E96E1350EF1406E1EA6A2F0E1224D5
:10127800E96E131CEF16D8901200166E0F0E131499
:10128800176E1338070B186E020A02E0186629D089
:10129800080E1502F3501424196E175206E0D89060
:1012A80019341B6E1750FADD16D0020E186209D0D9
:1012B80001EE00F0D8901934E926090EEE6EEE6AB8
:1012C8000AD0186608D001EE00F0D8901934E92643
:1012D800010EEE6EEE6AEA6A980E1524E96E165053
:1012E800EF1212000B500924E96E0C500A20EA6E26
:1012F800EFCF11F011AC26D011AA21D00D4C1ED081
:101308000BC012F00CC013F0122A000E1322125058
:101318000E6205D013500F6202D0126A136A12507F
:101328000924E96E13500A20EA6EEFCF10F0030E7D
:10133800106403D0100E10640CD0FF0C000C060EC5
:10134800106E07D011AA03D0040E106E02D0020E40
:10135800106E116A0B500924E96E0C500A20EA6ECF
:10136800EF50111A0B2A000E0C220B500E6205D0FA
:101378000C500F6202D00B6A0C6A1004126E1252E3
:1013880023E00D060DBE02D00D52D8B4000C0B5050
:101398000924E96E0C500A20EA6EEFBEFF0C0B50D0
:1013A8000924E96E0C500A20EA6EEF50111A0B2A34
:1013B800000E0C220B500E6205D00C500F6202D0AA
:1013C8000B6A0C6A1206DBD7113C02D010501200CF
:1013D800FF0C166E1338030B176E19B23CD0199414
:1013E80015BC19841F0E1516175005E0010A10E0E8
:1013F800030A23E02FD019A405D016501426000E96
:1014080015225ED0D89016301426000E152258D01A
:10141800158A158819B405D016501426000E152201
:101428004FD0D89016301426000E1522010E16162D
:1014380016501588D8B4159843D0158AD890163008
:101448001426000E1522010E161616501588D8B44B
:10145800159836D0120078B012003F0E15161750A6
:1014680005E0010A0EE0030A1DE029D0159615B81B
:101478001586159815BA1588100E13BC151A159AE5
:101488001FD0159615B81586080E13BC151A1588A1
:1014980019B006D0159A158615A812D0159610D031
:1014A800158A0ED0D88015AED890153214321598FA
:1014B800D8B01588158A080E13BC151A01D0120069
:1014C800D89014361536D8901432186A6950E96ED7
:1014D800020E6A24EA6EB00E1710EE6E18509EDBEC
:1014E800186E6950E96E020E6A24EA6E14C0EFFFA6
:1014F800185094DB186E6950E96E020E6A24EA6E81
:1015080015C0EFFF18508ADB186E6950E96E020E9D
:101518006A24EA6E181CEF6E000E80DB140EB4D439
:1015280008500914FF0AD8B4120010EEB0F00D6A82
:10153800080E0D6038D0E6CF0AF0E6CF0BF00BAE00
:1015480030D00BAC2ED0070E0B1624EE00F0200E78
:101558000D02F350D926106A010E0E6E0E5221E0CC
:10156800DFCF0CF00C38030B13E108500A6210D0DF
:1015780009500B620DD001EE80F06550E9262690E7
:10158800EFBA26803F0E0D24246E0E501BEC10F08F
:10159800040ED926102A0A2A000E0B22D8900E36DD
:1015A800DDD70D2AC5D712001C6ED9CF21F0DACFAE
:1015B80022F024EE00F0200E1B02F350D926040E70
:1015C8001A02F350D926DECF1EF023B01DD01E38E4
:1015D800030B1962E2D0195005E123A2DED0239251
:1015E80023B42382269023B22680370E1B24246E30
:1015F8001C501BEC10F0EA6A470E1B24E96E1C50C5
:10160800EF12140E41DCC9D01966C7D023A2C5D089
:101618001AB007D0EA6A980E1B24E96E1C1CEF1654
:1016280008D0EA6A980E1B24E96ED8901C30FF0A8D
:10163800EF161AB027D0268023B42690370E1B2425
:10164800246E1C501BEC10F0268023B426902F0E1D
:101658001B24246E1C501BEC10F0269023B426800B
:10166800370E1B24246ED8901C341BEC10F02690E7
:1016780023B426802F0E1B24246ED8901C341BEC18
:1016880010F07FD023B41FD02690370E1B24246E71
:101698001C501BEC10F026902F0E1B24246E1C509F
:1016A8001BEC10F02690370E1B24246ED8901C30AB
:1016B8001BEC10F026902F0E1B24246ED8901C30A3
:1016C8001BEC10F05ED0DFCF1FF01F5006E0050ABC
:1016D80004E00F0A02E0050A27E126901FB22680DF
:1016E800370E1B24246E1C501BEC10F026901FB2E2
:1016F80026802F0E1B24246E1C501BEC10F0269005
:101708001FB02680370E1B24246ED8901C301BEC8B
:1017180010F026901FB026802F0E1B24246ED89020
:101728001C301BEC10F02DD02680370E1B24246EA5
:101738001C501BEC10F02680370E1B24246ED8900A
:101748001C301BEC10F0040ED95E5F0EDF1417E09E
:10175800060E1A14206E080E1B02F35020241D6E6C
:1017680001EE00F0D8901D34E926010EEE6EEE6A07
:10177800EA6A980E1B24E96ED8901C30EF12040E0A
:10178800D9261BC024F0EA6A2F0E1B24E96EEF50FD
:1017980000EC10F0140E48EC07F021C0D9FF22C06D
:1017A800DAFF1200086E1EDA01EE80F06550E926B5
:1017B800D890EF340F6E16DA01EE80F06550E92606
:1017C8000F0EEF14106ED89010320F3201EE80F029
:1017D8006550E9261590EFBC15800850020A05E00F
:1017E800030A08E0010A19E02DD015B02ED00F68C1
:1017F8001068FF0C15B029D0EFBA02D0EFA804D0BA
:10180800EFAA05D0EFA803D00F681068FF0CEFAA65
:1018180002D0EFA8EF88EF8C18D015A003D00F687E
:101828001068FF0CF80E0F5C030E10580EE3FC0E48
:101838000F5C030E105809E20FC016F010C017F025
:10184800ADD903D00F681068FF0C10EEB0F0096A2C
:10185800080E09609AD1E6CF11F0E6CF12F012BE59
:1018680092D124EE00F0200E0902F350D926DD5063
:10187800159612BA1586159A12BC158A070E1216F5
:101888000E6A0850010A06E0010A04E0020AD8B408
:10189800D7D079D1010E0D6E0D52D8B474D1DCCFEA
:1018A8000BF00F50116242D0105012623FD001EE7F
:1018B80080F06550E9261592EFB8158201EE80F0A8
:1018C800E9261594EFBA1584086604D0040EDFBE25
:1018D800151A03D0020EDFBE151A15B616D015AAB2
:1018E80014D00EA012D008C019F0239015B623808A
:1018F800239215B22382238415B423940EC01AF0C0
:1019080009C01BF00D5050DE11D008C019F023900B
:1019180015B62380239215B22382239415B4238409
:101928000EC01AF009C01BF00D503EDE030ED9267A
:10193800DFAE77D0300EDF140C6E0C38086271D031
:10194800070EDD14146EDECF13F00F50136269D04A
:101958001050146266D001EE80F06550E9261592A9
:10196800EFB8158201EE80F0E9261594EFBA1584D8
:10197800086607D0040EDFBC151A159C15B4158C23
:1019880006D0020EDFBC151A159C15B2158CD8901E
:101998000B32D8900B32030E0B14010A05E0030A30
:1019A80006E0010A06E03DD015BC03D03AD015BCCC
:1019B80038D0D8900B32D8900B32030E0B160B5040
:1019C80007E0010A02E0030A2CE1159215B415821A
:1019D80015B616D015AA14D00EA012D008C019F04A
:1019E800239015B62380239215B22382238415B43D
:1019F80023940EC01AF009C01BF00D50D5DD11D08C
:101A080008C019F0239015B62380239215B22382BB
:101A1800239415B423840EC01AF009C01BF00D508E
:101A2800C3DD0E2A112A000E122215AA06D015B6F9
:101A380004D00EA002D01106125AD8900D362CD719
:101A4800010E0D6E0D52D8B49ED00F5011622CD0DD
:101A58001050126229D001EE80F06550E926EFAAF5
:101A680003D00E2AD8900D3601EE80F06550E92695
:101A78001592EFB81582020EDFBE151A08C019F0CC
:101A88002390239215B2238223940EC01AF009C022
:101A98001BF00D5089DD01EE80F06550E926EFAAB4
:101AA80003D00E06D8900D321598DCCF0BF0030E3C
:101AB800D926000EDA22DFAE5CD0300EDF140C6EB1
:101AC8000C38086256D00F0EDD14146EDECF13F0FA
:101AD800D890143213320F5013624BD01050146246
:101AE80048D0DD5001EE80F06550E926EFBA03D00A
:101AF800DEA003D03ED0DEA03CD001EE80F06550E1
:101B0800E9261592EFB81582020EDFBC151AD89097
:101B18000B32D8900B32030E0B14010A05E0030AAE
:101B280006E0010A06E025D015B203D022D015B28E
:101B380020D0D8900B32D8900B32030E0B160B50D6
:101B480005E0010A07E0030A05E013D0159415B271
:101B5800158415820BC019F02390239215B22382A5
:101B6800239415B423840EC01AF009C01BF00D503D
:101B78001BDD0E2AD8900D36157815B896D7112A80
:101B8800000E12225FD7092A63D60F5012002AD8F6
:101B9800C2A503D078820A0E756E1200C2A721D0A2
:101BA80001EE80F06550E926EFB81BD0030E16143D
:101BB800196ED890193601EE80F06550E926EFBA13
:101BC8001980080E19600DD0E26AD8901934B10F47
:101BD800E16EE7AE06D0EA6A470E1924E96EEE68B0
:101BE8007880120001EE80F06550E926EF6A652AD8
:101BF800600E656201D0656A12006750E96E020ED8
:101C08006824EA6EEF6A672A000E6822676605D0C4
:101C1800020E686202D0676A686A12001A6E69501A
:101C2800E96E020E6A24EA6EEF501A1A692A000E4B
:101C38006A22696605D0020E6A6202D0696A6A6A17
:101C48001A501200B00E126E136A146AB50E156E91
:101C580045DA116A106A040E10600ED0136E115026
:101C6800126E400E1124146EB50E156A152236DA5E
:101C7800400E1126102AEFD7D0DA268C01DB269CDD
:101C88001200B0DFC2A31200ADDF01EE80F0655094
:101C9800E9267C0EEF626FD0A5DF01EE80F065507B
:101CA800E926EFCF0CF09EDF9DDF01EE80F0655056
:101CB800E926EFCF09F096DF01EE80F06550E926BE
:101CC800D890EF34086ED88009AED890093208321F
:101CD8003F0EC0150B6EC1C00AF078B406D008508C
:101CE8000A6249D009500B6246D07CDF7BDFFC0ECC
:101CF8000C14200A0BE0080A09E0040A15E04C0A53
:101D080021E0080A1FE00C0A2AE035D078A409D09F
:101D1800C2AF07D00CC00DF008C00EF009C00FF01C
:101D28002BD8010E89D827D078B407D00CC00DF075
:101D380008C00EF009C00FF01FD8C2AF1CD07F0E2C
:101D48007BD819D078A406D0D1D8C2AF14D0400E11
:101D580073D811D0C2AF0FD0000E6ED80CD078B4A3
:101D680006D0C4D8C2AF07D0400E66D804D0C2AFE0
:101D780002D0000E61D8120015EE00F0E70EE66EF4
:101D88000E0EE66E7C0EE66E0DC0E6FF100EE66ED9
:101D9800D8900E360F36D8900E320FC0E6FF0EC020
:101DA800E6FFE66A166A01EE80F06550E926EFCF95
:101DB80014F014C018F018380F0B186E13DF01EE6A
:101DC80080F06550E926EFCF15F015C017F0179E83
:101DD80014B0178E18500FE1160E17600CD0B00E05
:101DE8001724E96E000E1820EA6EEFCF16F0140ED5
:101DF80048EC07F013D0160E175C010E18580EE2C7
:101E0800160E175E000E185A1750E96E040E1824A5
:101E1800EA6EEFCF16F0140E48EC07F0149216BED7
:101E2800148214C0E6FF15C0E6FF7F0E1614E66E96
:101E3800E66AE66A788A12000D6E0E6A6950E96EE3
:101E4800020E6A24EA6EB40EEE6E0E50E7DE0E6ED7
:101E58006950E96E020E6A24EA6E6F0EEF6E0E503C
:101E6800DDDE0E6E6950E96E020E6A24EA6E0DC060
:101E7800EFFF0E50D3DE0E6E6950E96E020E6A2433
:101E8800EA6E0E1CEF6E000EC9D6096AABDE01EED3
:101E980080F06550E9266F0EEF6227D078AA25D02A
:101EA800789A15EE00F06950E96E020E6A24EA6E1F
:101EB800E6CFEFFF0950B2DE096E020EE75C086E4E
:101EC8006950E96E020E6A24EA6EE6CFEFFF095008
:101ED800A5DE096E082EF4D76950E96E020E6A2451
:101EE800EA6E091CEF6E000E99D6120001EE80F022
:101EF8006550E926EFCF0FF075DE01EE80F06550F2
:101F0800E926EFCF0EF00E9E0FB00E8E6BDE01EEBF
:101F180080F06550E926EFCF0DF00D9E0FB20D8EC3
:101F28000F380F0B0F6E140E0E6202D00F5205E021
:101F3800150E0E620BD00F6609D0AA0E0D6201D0E5
:101F480081DEA10E5E6E140E48EF07F00F5013E10C
:101F5800140E0E6010D0B00E0E24E96E000E0F2085
:101F6800EA6E0DC0EFFF04000EC019F00FC01AF0A2
:101F78000D5078D81BD0160E0E5C010E0F5815E2C6
:101F8800160E0E5E000E0F5A0E50E96E040E0F2448
:101F9800EA6E0DC0EFFF0400400E0E24196E000E0D
:101FA8000F201A6E0D505ED801D0120036D90F508E
:101FB8000AE1100E0E6007D0010E0E14010A03E1AB
:101FC800268C5ED9269C510E5E6E140E48EF07F0E3
:101FD800196EF00E801619508026899881CF1AF054
:101FE8001A9082BA1A808988EA6A900E1924E96ED2
:101FF800EF501A1A1A501200256EEA6A900E24241D
:10200800E96EEF50251A010E9316949A25C081FFA8
:1020180025A0829A25B0828AF00E8016080E242404
:10202800802689988988FE0E9312948A1200256E5C
:1020380024C0E9FFEA6AD890EF14D8A4D88026A073
:1020480003D02550EF1202D0251CEF161200A6B2BD
:10205800FED71CC0A9FF1DC0AAFFA69EA69CA680ED
:10206800A85012001B6E19C01CF01AC01DF0EFDF3B
:102078001B1832E0A6B2FED71BC0A8FF19C0A9FFE3
:102088001AC0AAFFA69EA69CA684F29E550EA76E0D
:10209800AA0EA76EA682F28EA694632A000E642268
:1020A800E90E635C030E64580EE3636A646A612A8E
:1020B800000E6222F10E615C030E625804E3400ECA
:1020C800616E010E626E19C01CF01AC01DF0BFDFF0
:1020D8001B1802E0D8901200D8801200A68EA69C89
:1020E800F86A1550F76EC00E1414F66E12C0E9FFA8
:1020F80013C0EAFF400E166E0900F552F5CFEEFF49
:10210800162EFAD712000AC0F6FF0BC0F7FFF86ABE
:10211800A68EA69C0800F55012000F0EC16E070E81
:10212800B46E300E806EC00E926E816A9368D50EC2
:10213800826EEA0E946ED0A60AD0D0A408D000EE23
:1021480000F00F0EEE6AEA62FDD7E9AEFBD7F19C0C
:10215800F298F2924A0EAF6EAC84AC98AB8E9D9812
:102168009D9AAB98D56A800ECD6E9E909D80490E43
:10217800CA6ECC6A7C0ECB6E9E929D82B16A1200AA
:10218800572A582A592A592A5A2A5B2A140E0A6E9B
:10219800B50E0B6EB8DF096E140E1C6E1D6A57DF84
:1021A800091809E009C0A8FFA684550EA76EAA0E53
:1021B800A76EA682A69400EEB0F0076A086AA68405
:1021C80007C01CF008C01DF042DFEE6E550EA76E6A
:1021D800AA0EA76EA682072A000E0822085003E15D
:1021E800150E0764EDD704EE00F0400E076E086A7E
:1021F80007C01CF008C01DF02ADFEE6E550EA76E52
:10220800AA0EA76EA682072A000E0822400E075CB7
:10221800010E0858EDE3A69412006068010E126ED4
:1022280010EEB0F0136A080E136029D0EA6A900E17
:102238001324E96EEF6A010E156E24EE00F0200EED
:102248001302F350D926E650E6BE03D0D92A121C51
:102258006016176A200E17600ED0DFAE06D0EA6A45
:10226800900E1324E96E1550EF12D8901536040E0F
:10227800D9261726EFD7D8901236132AD4D71200AA
:10228800010E9316949A60C081FF60A0829A60B094
:10229800828A899A898AFE0E9312948A8B981C6E78
:1022A800030E1D6ED4DE616E1C68030E1D6ECFDE3C
:1022B800626E1890F10E615C030E625805E3188097
:1022C800400E616E010E626E269AC2B1268A26AA57
:1022D80015D026AC05D061C016F062C017F005D045
:1022E8006128166E000E6220176EF10E165C030E42
:1022F800175804E3400E166E010E176E070E126E85
:1023080012BE74D0E26AD8901234B10FE16E26AAD8
:1023180060D018B002D026AC02D0136A0AD012508E
:1023280061241C6E000E12BEFF0E62201D6E8FDE31
:10233800136E040012501624196E000E12BEFF0E02
:1023480017201A6E13508EDEE7BE3DD0EA6A370EAC
:102358001224E96E13C0EFFFE7AA2FD0EA6A2F0E06
:102368001224E96E13C0EFFF12C024F0EA6A2F0EA0
:102378001224E96EEF5040DE020E156E010E146E47
:10238800080E146026D0030E1314030A0BE1196A11
:1023980023802382238414C01AF012C01BF0155026
:1023A800D8EC0AF0D8901332D8901332D89015365A
:1023B800D8901536020E1426E3D7EA6A470E12247F
:1023C800E96EEE6806D0EA6A3F0E1224E96E13C081
:1023D800EFFFE7AE09D01250FBDD136EEA6A370E45
:1023E8001224E96E13C0EFFF12068AD716C061F0F7
:1023F80017C062F00400FE0E196E030E1A6E6150CB
:0E24080031DE04001968030E1A6E62502BD6E6
:10B50000008008801080188020802880308038805B
:06B51000E71007000557DB
:10B54000230000002300000023000000230000006F
:10B55000230000002300000023000000230000005F
:10B56000230000002300000023000000230000004F
:10B57000230000002300000023000000230000003F
:10B58000230000002300000023000000230000002F
:10B59000230000002300000023000000230000001F
:10B5A000230000002300000023000000230000000F
:10B5B00023000000230000002300000023000000FF
:10B5C00023000000230000002300000023000000EF
:10B5D00023000000230000002300000023000000DF
:10B5E00023000000230000002300000023000000CF
:10B5F00023000000230000002300000023000000BF
:10B6000023000000230000002300000023000000AE
:10B61000230000002300000023000000230000009E
:10B62000230000002300000023000000230000008E
:10B63000230000002300000023000000230000007E
:0200000400F00A
:100000000080088010801880208028803080388010
:06001000E7100700055790
:100040002300000023000000230000002300000024
:100050002300000023000000230000002300000014
:100060002300000023000000230000002300000004
:1000700023000000230000002300000023000000F4
:1000800023000000230000002300000023000000E4
:1000900023000000230000002300000023000000D4
:1000A00023000000230000002300000023000000C4
:1000B00023000000230000002300000023000000B4
:1000C00023000000230000002300000023000000A4
:1000D0002300000023000000230000002300000094
:1000E0002300000023000000230000002300000084
:1000F0002300000023000000230000002300000074
:100100002300000023000000230000002300000063
:100110002300000023000000230000002300000053
:100120002300000023000000230000002300000043
:100130002300000023000000230000002300000033
:020000040020DA
:080000000507000100010001E9
:020000040030CA
:08000000FF021F08FF8181FFD0
:00000001FF
